:103800000C94241C0C94411C0C94411C0C94411CE1
:103810000C94411C0C94411C0C94411C0C94411CB4
:103820000C94411C0C94411C0C94411C0C94411CA4
:103830000C94411C0C94411C0C94411C0C94411C94
:103840000C94411C0C94411C11241FBECFE5D4E004
:10385000DEBFCDBF10E0A0E6B0E0E2EFFEE302C0C5
:1038600005900D92A036B107D9F711E0A0E6B0E0BF
:1038700001C01D92A43AB107E1F70E94301F0C94D9
:10388000771F0C94001C0F92AF93BF93CF93DF93DD
:10389000EF93FF93FC01EA01DB01C8950992319691
:1038A0001197D9F7FF91EF91DF91CF91BF91AF9130
:1038B0000F9008950F921F920F931F93AF93BF9392
:1038C000CF93DF93EF93FF93FC01EA01DB0110E854
:1038D0000990199001E04CD03296129711F01250D5
:1038E000B9F7FC0103E044D005E042D000E810E065
:1038F000800F911F109759F7FF91EF91DF91CF91B2
:10390000BF91AF911F910F911F900F9008950F934A
:103910001F93EF93FF93FC0103E02AD000E810E02F
:10392000E00FF11FE617F707B9F7FF91EF911F912D
:103930000F9108950F930F9222D0082E09E018D00E
:103940000F900F9108950F930F92EF93FF9317D05D
:10395000FC0160935700C895802DFF91EF910F9067
:103960000F9108950F930BD001E102D00F910895AC
:10397000E199FECF00935700E895FFFF000000910A
:10398000570000FDFCCF089583E089B98AB18861B2
:103990008AB908958AB1877E8AB908958CB95E9BE9
:1039A000FECF5E9A08958CB108958BB1807808950A
:1039B000AC0120E030E009C05F9BFECF8CB1FA0182
:1039C000E20FF31F80832F5F3F4F26173707A0F3C7
:1039D00081E00895FC0120E030E008C080818CB9CE
:1039E0005E9BFECF31965E9A2F5F3F4F26173707BB
:1039F000A8F381E00895813879F0823818F480388E
:103A000039F408C0823851F0883911F483E0089500
:103A100080E0089582E0089581E0089582E10895AC
:103A20006091A0007091A1004091A2015091A3016A
:103A300020E030E010C0C901840F951F9FBB8EBBF2
:103A4000F901EE55FF4F80818DBBE29AE19AE19931
:103A5000FECF2F5F3F4F2617370768F3460F571FDC
:103A60005093A3014093A20108956091A00070912A
:103A7000A1004091A2015091A30120E030E00DC0CF
:103A8000C901840F951F9FBB8EBBE09A8DB3F901CE
:103A9000EE55FF4F80832F5F3F4F2617370780F388
:103AA000460F571F5093A3014093A201089540E091
:103AB00050E00BC020E030E000002F5F3F4F63E09C
:103AC0002B363607C9F74F5F5F4F4817590790F3FA
:103AD00008956091A0007091A1008091A201909141
:103AE000A30142EA50E0880F991F0E94431C0895E9
:103AF000CF93DF93C0E0D0E011C0AE014E555F4FD1
:103B00008091A2019091A301880F991F60E870E055
:103B10008C0F9D1F0E945A1CC058DF4F8091A0003F
:103B20009091A100C817D90740F30E94B21CDF9101
:103B3000CF9108950E94D51C8823E1F30E94D31CE5
:103B4000803211F481E0089585E10E94CE1C80E06E
:103B50000895DF92EF92FF920F931F93CF93DF931D
:103B600069E081E090E00E94A31C84FF03C08F7E87
:103B70000E949A1CDD240E94D51C8823E1F30E9438
:103B8000D31C8235C0F4803508F078C0813409F444
:103B900043C0823448F4813321F1803409F452C1A6
:103BA000803309F04BC16AC0823409F458C08534AF
:103BB00009F044C157C0863509F40DC1873538F482
:103BC000823509F461C0853509F038C16CC084378D
:103BD00009F4A6C0853709F4EEC0843609F02EC179
:103BE0007AC00E949A1D882331F284E10E94CE1C83
:103BF00081E40E94CE1C86E50E94CE1C82E50E94D4
:103C0000CE1C80E20E94CE1C83E50E94CE1C84E57F
:103C10000E94CE1C8BE40EC161E070E080E690E073
:103C20000E94D81C0E949A1D882309F4A4CF84E125
:103C30000E94CE1C80916000813869F0823818F4AF
:103C4000803839F4C6C0823841F0883911F483E0F5
:103C5000F1C080E0EFC081E0EDC082E1EBC064E143
:103C600070E008C061E070E080E690E00E94D81C3F
:103C700064E070E080E690E00E94D81C0E949A1DEB
:103C8000882309F478CF0DC00E949A1D882309F477
:103C900072CF60E070E480E090E00E94871C0E9498
:103CA000B21C84E1C7C062E070E080E690E00E9450
:103CB000D81C0E949A1D882309F45DCFF090610002
:103CC000EE24809160009701280F311D3093A301ED
:103CD0002093A201E6CF63E070E080E690E00E94CE
:103CE000D81CD0916000C0E080916100BE01680FD7
:103CF000711D7093A1006093A00082EA90E00E9481
:103D0000D81C0E949A1D882309F435CF8091620047
:103D1000863419F40E94781DC4CF0E94101DC1CFB3
:103D200063E070E080E690E00E94D81C1091600093
:103D300000E0809161009801280F311D3093A100AF
:103D40002093A0000E949A1D882309F414CF80912B
:103D50006200863459F04091A0005091A10060911A
:103D6000A2017091A30120E030E010C00E94691D03
:103D700016C0C901860F971F9FBB8EBBE09A8DB3FB
:103D8000F901EE55FF4F80832F5F3F4F2417350712
:103D900080F3460F571F5093A3014093A20184E183
:103DA0000E94CE1C6091A0007091A10082EA90E078
:103DB0000E94EA1C41C00E949A1D882309F4DBCEB0
:103DC00084E10E94CE1C8EE10E94CE1C84E90E94F8
:103DD000CE1C82E02FC064E070E080E690E00E949C
:103DE000D81C0E949A1D882309F4C5CE84E10E9444
:103DF000CE1C80916000803531F480916100882371
:103E000059F4DD2412C0883581F480916100883036
:103E100041F453E0D52E09C0883039F442E0D42E65
:103E200004C0882311F4DD24D39469E08D2D90E043
:103E30000E94A31C0E94CE1C80E101C085E10E946B
:103E4000CE1C99CEDF91CF911F910F91FF90EF90F3
:103E5000DF9008950E94CA1CE0E0F0E00995089503
:103E60001F93F894E199FECF8EEF91E09FBB8EBB3C
:103E7000E09A8DB3843B99F4E199FECF8FEF91E006
:103E80009FBB8EBBE09A8DB3833C49F4E199FECF92
:103E90008DEF91E09FBB8EBBE09A8DB381BF0E94F6
:103EA000C41C0E94D31C1EE119C00000019643E00F
:103EB0008B369407D1F72F5F3F4F2436310519F029
:103EC00080E090E0F2CF0E94D51C882319F00E9478
:103ED000A91D07C0115018BB112319F020E030E0D4
:103EE000EFCF0E942A1F80E090E01F910895F89480
:023EF000FFCF02
:0400000300003800C1
:00000001FF
